:0E1F5500010204080001020203030404050552
:10067500E4F513F512F511F510C260C23DC258C27A
:10068500411209BE7E0F7FB88E3F8F4075470F75AB
:1006950048CA753D0F753ED475450F7546FC754CBA
:1006A50010754D2490E680E030E70E853D41853E8E
:1006B50042854543854644800C85454185464285AE
:1006C5003D43853E44EE54E070030207E675140091
:1006D5007515807E0F7FB88E168F17C374529FFFD6
:1006E50074109ECF2402CF3400FEE48F0F8E0EF5DA
:1006F5000DF50CF50BF50AF509F508AF0FAE0EADC6
:100705000DAC0CAB0BAA0AA909A808C3121D03500E
:100715002AE515250BF582E514350AF58374CDF028
:10072500E4FAF9F8E50B2401F50BEA350AF50AE9CF
:100735003509F509E83508F50880C0E4F50BF50A33
:10074500F509F508AF0FAE0EAD0DAC0CAB0BAA0A53
:10075500A909A808C3121D035035AE0AAF0BE5174A
:100765002FF582E5163EF583E0FDE5152FF582E5CB
:10077500143EF583EDF0E4FAF9F8EF2401F50BEA00
:100785003EF50AE93509F509E83508F50880B58526
:10079500143F85154074B82480FF740F34FFFEC3E1
:1007A500E5489FF548E5479EF547C3E5429FF54275
:1007B500E5419EF541C3E5449FF544E5439EF54378
:1007C500C3E53E9FF53EE53D9EF53DC3E5469FF5F8
:1007D50046E5459EF545C3E54D9FF54DE54C9EF532
:1007E5004CD2E843D82090E668E04409F090E65CF6
:1007F500E0443DF090E65EE04408F0D2AF120863B5
:1008050090E680E020E105D261121A2690E680E0AC
:1008150054F7F0538EF8C26030410512038EC24181
:10082500306029121FA35024C260121C3D203D16C2
:1008350090E682E030E704E020E1EF90E682E030E8
:10084500E604E020E0E4121A83121FA5120D9C12A3
:0D0855000D9C120D9C120D9C120D9C80BB81
:010862002273
:10038E0090E6B9E070030204B7147003020560240E
:10039E00FE70030205F524FB70030204B114700312
:1003AE000204AB14700302049F1470030204A5240C
:1003BE00056003020661121FA7400302066D90E658
:1003CE00BBE024FE603E14700302046624FD601F31
:1003DE0014605B24066003020495E53F90E6B3F0DB
:1003EE00000000E54090E6B4F000000002066DE566
:1003FE004790E6B3F0000000E54890E6B4F0000048
:10040E000002066D90E680E030E708853D41853EAE
:10041E00428006854541854642E54190E6B3F000AF
:10042E000000E54290E6B4F000000002066D90E692
:10043E0080E030E7088545438546448006853D4388
:10044E00853E44E54390E6B3F0000000E54490E6B7
:10045E00B4F000000002066D90E6BAE0FF121AAF8B
:10046E00AA06A9077B01EA496013EE90E6B3F000F5
:10047E000000EF90E6B4F000000002066D90E6A0DA
:10048E00E04401F002066D90E6A0E04401F00206A1
:10049E006D121EDF02066D121F8202066D12000320
:1004AE0002066D121ECD02066D121FA94003020632
:1004BE006D90E6B8E0247F602B14603C240260034C
:1004CE00020556A23DE433FF25E0FFA258E4334F68
:1004DE0090E740F0E4A3F090E68AF090E68B740289
:1004EE00F002066DE490E740F0A3F090E68AF090FB
:1004FE00E68B7402F002066D90E6BCE0547EFF7E41
:10050E0000E0D3948040067C007D0180047C007D59
:10051E0000EC4EFEED4F2459F582741F3EF583E438
:10052E0093FF3395E0FEEF24A1FFEE34E68F82F5C4
:10053E0083E0540190E740F0E4A3F090E68AF09057
:10054E00E68B7402F002066D90E6A0E04401F00224
:10055E00066D121FAB400302066D90E6B8E024FE56
:10056E00601D2402600302066D90E6BAE0B4010538
:10057E00C23D02066D90E6A0E04401F002066D90C9
:10058E00E6BAE0705990E6BCE0547EFF7E00E0D300
:10059E00948040067C007D0180047C007D00EC4E42
:1005AE00FEED4F2459F582741F3EF583E493FF331D
:1005BE0095E0FEEF24A1FFEE34E68F82F583E05442
:1005CE00FEF090E6BCE05480FF131313541FFFE0BF
:1005DE00540F2F90E683F0E04420F002066D90E673
:1005EE00A0E04401F08078121FAD507390E6B8E0A1
:1005FE0024FE60202402706790E6BAE0B40104D2B3
:10060E003D805C90E6BAE06402605490E6A0E0445F
:10061E0001F0804B90E6BCE0547EFF7E00E0D39468
:10062E008040067C007D0180047C007D00EC4EFE47
:10063E00ED4F2459F582741F3EF583E493FF3395F5
:10064E00E0FEEF24A1FFEE34E68F82F583E0440155
:10065E00F0800C121FAF500790E6A0E04401F0901E
:06066E00E6A0E04480F06C
:010674002263
:03003300021F9F0A
:041F9F0053D8EF32F2
:101F3600040103000505000301000200FFFFFEFE89
:1009BE0090E682E04410F090E600E054E74410F038
:1009CE00D23D12147190E61274E2F01214CC90E63D
:1009DE001074A0F090E611F0000000E490E68DF0A7
:1009EE00000000F58690E601E04402F075B2FF7556
:1009FE00B4EF75B5FF75B6FF75A0E0E4F5B17C00F8
:100A0E00EC90E606F090E6077456F090E605E044AA
:100A1E0006F0758C06E58954F84402F589538EF775
:100A2E00D28CD2A9752460908003E524F0C2817522
:100A3E00B2FD308104D2438002C243304307AF601F
:100A4E00121A558005AF60121CAAD2068520B17508
:100A5E005B40D24875230175217775227F7525037A
:100A6E00908000E521F0908001E522F0908002E573
:100A7E0023F0908004E525F0908010E526F090E0BC
:100A8E00917401F07D0C7F401219F6E4FD7F701217
:100A9E0019F67DD8E4FF1219F67D407F101219F673
:100AAE00D24E7D0C7F201219F67D327F501219F630
:0F0ABE007D1E7F301219F67D327F601219F622ED
:100863007F01121B80E4F55A90E092F0A3F07531FA
:1008730002E5312410FD7FA0121C8690E093E02F47
:10088300F090E092E03400F00531E531C39420406C
:10089300E07D107FA0121C8690E093E02FF090E0A3
:1008A30092E03400F07D117FA0121C86EFFE90E0F1
:1008B30093E02400F090E092E03EF0E0F47003A3B4
:1008C300E0F470417D157FA0121C868F5A7D167F40
:1008D300A0121C868F327D1A7FA0121C868F337D57
:1008E300247FA0121C868F317D227FA0121C868F4D
:1008F30034E53113923AE531A2E29250C413135412
:100903000390E08EF0E4F54EE55A14601014601F76
:1009130014602114602E8000755218803775523090
:10092300E53130E1047F0280027F018F4E8025751F
:1009330052108020755246754E01D22D908004E5E9
:1009430025F0801075526B754E03D22D908004E50F
:1009530025F0D242204203E4F534E4F531E533C314
:1009630094804003753101E5312450FFE53325E0E0
:10097300FD1219F6E4F531E532C394804003753175
:1009830001E5312460FFE53225E0FD1219F6E4F5B7
:1009930033F532A23A922A908004E525F012000E34
:1009A300121809121F03304309121D9490E0A5EF9A
:0B09B300F02212195B90E0A5EFF0228B
:100CB900304307121D948F3A800512195B8F3A2031
:100CC9005903020D6BE4FD90E0A5E0FCC3953A40A1
:100CD900027DFFE538547FFFBF0417ED600C90E0FB
:100CE9008AE0F4600DE004F0800890E08AE0600298
:100CF90014F0E5385407707CED6030ECC3953AF593
:100D090019E49400F518E519AE187803C333CE3306
:100D1900CED8F9F5198E1890E08AE0FB7E002519E6
:100D2900EE35187039EB2519FD8033ECFFE53AC330
:100D39009FF519E49400F518E519AE187803C33343
:100D4900CE33CED8F9F5198E1890E08AE0FFFBC3AF
:100D5900E5199BE51894005005C3EF9519FD8D60C1
:100D6900801290E08AE0600CE53854077006E5606F
:100D790060021560304307AF60121A558005AF60F5
:100D8900121CAA30420AE5607004D2808002C28037
:020D9900C25541
:010D9B002235
:100D9C00305F3F90E780E0F531A3E0FFC4540FF5DE
:100DAC003BE531B4A509E53B901F3693B4FF051222
:100DBC001E0D801CE53B901F3693FF90E781E0549D
:100DCC000F6F6004EFB4FE051210E48003121F9A3B
:100DDC00C25F30562D854F55855056C3E54B955601
:100DEC00E54A95555006854A55854B56D3E556949C
:100DFC0000E55594014006755501755600121353C4
:100E0C0080031213B8304C0F120ACDA24A924A50EA
:100E1C0030C24CC24A802AE52F6026E54B2537FFAD
:100E2C00E54A3536FED3EF94FFEE940E5003304274
:100E3C000CD3EF94FFEE941E5007304204D24C15A5
:0B0E4C002F305506205E03120CB92267
:1014CC0000000090E6187404F0000000740CF000AA
:1014DC00000090E680E030E71090E6207402F00007
:1014EC000000E490E621F0800EE490E620F000008D
:1014FC000090E6217440F0000000E490E6CEF0008D
:10150C00000090E6CFF000000090E6D0F000000064
:08151C0090E6D1F0000000226E
:021FA300D32247
:021FA500D32245
:021FA700D32243
:0800030090E6BAE0F51BD322E0
:101ECD0090E740E51BF0E490E68AF090E68B04F095
:021EDD00D3220E
:081F820090E6BAE0F51AD32243
:101EDF0090E740E51AF0E490E68AF090E68B04F084
:021EEF00D322FC
:021FA900D32241
:021FAB00D3223F
:021FAD00D3223D
:021FAF00D3223B
:101DAD00C0E0C083C082D2415391EF90E65D7401D3
:081DBD00F0D082D083D0E032A7
:101E2500C0E0C083C0825391EF90E65D7404F0D0AA
:061E350082D083D0E032F0
:101E3B00C0E0C083C0825391EF90E65D7402F0D096
:061E4B0082D083D0E032DA
:10188100C0E0C083C08290E680E030E70E853D4134
:10189100853E42854543854644800C8545418546C4
:1018A10042853D43853E445391EF90E65D7410F0CF
:0718B100D082D083D0E032A9
:101DC500C0E0C083C082D2605391EF90E65D740895
:081DD500F0D082D083D0E0328F
:1018B800C0E0C083C08290E680E030E70E853D41FD
:1018C800853E42854543854644800C85454185468D
:1018D80042853D43853E445391EF90E65D7420F088
:0718E800D082D083D0E03272
:101DDD00C0E0C083C082D25F5391EF90E65F74087C
:081DED00F0D082D083D0E03277
:01005200327B
:100FB8001201000200000040970D0101010001022A
:100FC80000010A0600020000004001000902270093
:100FD800010100A0000904000003FF00000007054C
:100FE8008102400000070501024000000705820257
:100FF8000002000009022700010100A00009040006
:101008000003FF00000007058102400000070501FA
:1010180002400000070582024000000004030904A2
:101028000A035300420049004700200355005300BB
:10103800420046002D00430041004D0020004500BD
:0D1048006E00670069006E0065000000008A
:0A0EF500AE49C3E5389EC39F40F8E4
:010EFF0022D0
:10180900E490800DF0908006F0A3740AF0908008AF
:10181900E4F0A37409F090800AE4F0A304F0D22E56
:10182900908004E525F0C22F7F0A120EF5E525F018
:0C183900D22FE525F0120EF5121F6322DD
:10000E00908000E521F0908001E522F0908003E5DC
:10001E0024F0908002E523F0908003E524F0908098
:05002E0004E525F022AD
:101B8000E5A020E5047E0180027E008E31EF600535
:101B900053A0DF800743A020A23C9246E5317004A9
:071BA0007F0180027F00229B
:1011FC00C24890E785E0540CF531E030E42490E7E8
:10120C0083E0F55EA3E0F562E55B54F34404F55B23
:10121C00D251E5317043C251E55B54F34408F55BA0
:10122C00803790E782E0F530A3E0F535A3E0F53C9C
:10123C00E55B54FC4401F55BD253E531700AC253B3
:10124C00E55B54FC4402F55BA23C9246303C0AAF91
:10125C0038EF653860FB121E7DE531B40405D244CD
:10126C001217CAE531B40803121702D248121F959F
:01127C00224F
:10192600C24890E782E030E014E55B540C60205337
:101936005BF330511A121702435B0C8012E55B54BD
:1019460003600C535BFC305306121702435B03D251
:0519560048121F95225C
:10162100C2AF90E782E030E407E0A2E3925E803748
:10163100C25EC25990E783E090E0A5F090E782E0B6
:1016410030E10BA3E0F560E490E08AF0801990E7C7
:1016510082E030E00CD25990E784E090E08AF0809B
:0D1661000690E08A7401F0D2AF121F9522AE
:101BCE00E490E097F030590204F090E0A5E090E048
:101BDE0098F0A3E53AF0A37480F0A3E560F0753BAE
:051BEE0035121D582214
:101CCE00C2AF90E782E0F532A3E0F52DA3E0F53345
:101CDE00A3E0F52EC257A3E030E002D257D2AF12E6
:031CEE001F95221D
:1018450090E783E07032A3E0702E90E786E0C394C2
:10185500014025E0D39407501FE54EB40104E0B4E0
:101865000716E54EB4020890E786E0640460099027
:0B187500E786E0F55F120E57121F958A
:011880002245
:1018EF0090E782E02410547FF531E030E71690E75F
:1018FF0084E0FFAD31121C8690E097EFF0753B71DD
:10190F00121D582290E784E0FF90E783E0FBAD3192
:07191F00121C18121F952293
:10152400121F9590E782E0FFC454C0F53BE4F557E1
:10153400E53BB44004C2058015E53B7004D2058048
:101544000DE53BB4800575573F800375570FE55B88
:10155400543F453BF55B8520B190E782E05403F5A9
:101564003BB401031217CAE53BB40203121702E5A8
:081574003BB40303121F032224
:10127D00C2AFE55B54CF90E097F0305C04E04410D2
:10128D00F0305B0790E097E04420F0305A0790E093
:10129D0097E04430F090E0987401F0E5326004E09E
:1012AD004410F0E52D600790E098E04420F0E53320
:1012BD00600790E098E04440F0E52E600790E098DC
:1012CD00E04480F0E563540790E099F0205404E089
:0C12DD004408F0D2AF753B93121D58225C
:0C004600E490E097F0753BB1121D5822C9
:10174600121F95C23F90E782E030E002D23F90E759
:1017560082E054186023E5515403901F5593FFE52A
:101766002454F0FEEF4EF52490E782E030E40DD2EB
:101776003990E08FE539F080035324F0908003E53B
:0317860024F0222A
:0D003600070F0606070D1E0A07070A010A3C
:101D1400305404055180021551E5515403901F5568
:101D240093FFE52454F0FEEF4EF524908003E52460
:021D3400F0229B
:101F0300C24DC244755F06120E57755F07120E5716
:011F130022AB
:1017CA00C24D305A04D25D8033C25D305C2ED25B8A
:1017DA00C25CE5515403901F5593FFE52454F0FE73
:1017EA00EF4EF524908003E524F0E4F558F559E529
:0F17FA004EB402047F0280027F078F5DD24D2222
:10170200C24D305B04D2528038C252304733D25A73
:10171200C247C2078520B1E5515403901F5593FF7C
:10172200E52454F0FEEF4EF524908003E524F0E426
:10173200F558F559E54EB402047F0280027F078F07
:041742005DD24D2205
:03000B000200569A
:10005600C0E0C0F0C083C082C0D075D000C000C070
:0D00660001C002C003C004C005C006C007F1
:1000730090E089E004F0304615E030E011B208B2B8
:1000830009908000E521F0B208B209E521F090E083
:1000930089E0540F60030202490549304D76205B25
:1000A30003305A5D205A0CE559700890E08BE064E8
:1000B300097061E5587046121D14E54E6008E55954
:1000C300B40203D55D020559E55990003693F558FE
:1000D300E5596406703E305B16D247C25B30440478
:1000E300D207C2448520B130522A1217028025D28A
:1000F3005CC25AB254305D1C1217CA80171558805F
:1001030013E558600FD5580C2039095324F090801B
:1001130003E524F0303F129080007474F0751810DA
:10012300D518FD908000E521F090E08BE004F0E02D
:10013300640A6003020249F00538E53870020539A4
:10014300D2552048030201DAE55B5403FFBF0108DF
:10015300205C03304702055BE55B5403FFBF021DD0
:10016300AF3C153CEF7016AF351535EF700FAF3060
:100173001530EF7008305310121702055BE55B541E
:1001830003FFBF030E305C0B303C05C2461212E97D
:10019300535BFCE55B540CFFBF040C204703305C4E
:1001A300067404255BF55BE55B540CFFBF081AAFCF
:1001B300621562EF7013AF5E155EEF700C30511471
:1001C3001217027404255BF55BE55B540CFFBF0C4F
:1001D30006305C03535BF3305706E538540F703237
:1001E300751800E53260054318041532E52D6005E6
:1001F300431808152DE53360054318011533E52E23
:100203006005431802152EE52054F04518F52085A6
:1002130020B1E557600655387002B2058520B1302C
:100223003924205B21205A1EE564B5631990E08FC1
:10023300E0FFC3E5399FD39402400BC2395324F046
:10024300908003E524F090E089E0540F6408600394
:10025300020373204B03020373E5646563700302B7
:100263000373900036E493B5660EE564B40709534F
:1002730024F0908003E524F0AF661566EF60030277
:100283000373055CE55CB4010A90003EE493F566F4
:10029300020370E55CB4020990003FE493F56680C5
:1002A30028E55C64037027E564B4071630490AE562
:1002B30065B401057566788010900040E493F56697
:1002C3008007900041E493F566B254020370E55C45
:1002D30064067029F557C2058520B1856463A23889
:1002E3009254D24DE563640760030203737563029E
:1002F300756402C25AC25BC247D25C8073E55C6418
:10030300056045E56464077054204951E565D3945D
:1003130004504AE5515403FF90E08EE06F703E2095
:100323004926E54EB403057565018016E54EB40212
:100333000575650F800CE54E70047F0C80027F0409
:100343008F65D249B254801B2039095324F0908021
:1003530003E524F090003CE493F56680131565E50E
:100363006560F1755C0190003EE493F566121D141F
:10037300D007D006D005D004D003D002D001D000DE
:0B038300D0D0D082D083D0F0D0E03288
:100ACD00E56124F97003020B8C24076003020BCD42
:100ADD00204C03020BCDC2AFC22F908004E525F050
:100AED007F05121F90C22E908004E525F03042083C
:100AFD00D20B908000E521F0304E19303C0CC246EF
:100B0D0090E091E0FF121EF1801F90E091E0FF1246
:100B1D001C628015303A0A90E091E0FF121E518060
:100B2D000890E091E0FF121D7790E092E0FEA3E0C7
:100B3D00FF8E1CF51D90E08CE0FCA3E0FDEF2DFB7E
:100B4D00EE3CCB2537F51DEB3536F51C908006F0C8
:100B5D00A3E51DF0C39FF51DE51C9EF51C908008B7
:100B6D00F0A3E51DF090800AECF0A3EDF0D22E90ED
:100B7D008004E525F0D22FE525F0D2AF756107127F
:100B8D001F46503CE537254BF54BE536354AF54AC2
:100B9D00E52F6027E54B2537FFE54A3536FED3EFC8
:100BAD0094FFEE940E500330420CD3EF94FFEE946D
:100BBD001E5008304205152F020AE3E4F561D24AB2
:010BCD002205
:101B3000EE2F6020D3121DF5908001E5220EC2E544
:101B4000F0C2E3F06403F0D2E3F06403F0DFF2DE0E
:081B5000F0E522F0C3021DF5CF
:101D7700908001E522C2E5F0C2E3F06403F030E3AE
:0D1D870003C2E3F0D2E3F0DFF5E522F02225
:101E5100908001E522C2E4F06403C2E4F0D2E4F030
:061E6100DFF8E522F0228B
:101BF300EF2E601DD3121DF5908001E5220E6418AF
:101C0300F06403F06418F06403F0DFF2DEF0E52221
:051C1300F0C3021DF505
:101E6700908002E523D2E3F07805121F6FC2E3F0FA
:061E7700121990C23E2288
:10199000908001E5227D7D7C0B7B10C2AF6BF06CEB
:1019A000F06BF06CF06BF06CF06BF06CF06BF06C5B
:1019B000F06BF06CF06BF06CF06BF06CF0DDDED285
:0419C000AFD23E2242
:0A1F6F00D80008D8000800D8F722B7
:051F9000EFF8021F6FD5
:061F8A00F0780A021F6F4F
:101C6200908000E521304206D2E0C2E18007C2E066
:101C7200121F8A6403121F8A6403121F8ADFE6D2CC
:041C8200E0021F8AD3
:091F79007E007F557C0002141665
:10141600C246EE2F604E0ED3121DF5303C00908072
:1014260000E521304204C2E18007C2E0121F8A644F
:1014360003121F8A6403121F8A203CF5D2E0121F92
:101446008AEFBE0105C3940440045CB40112C312C2
:101456001DF5A9527840121F6FD9F9DFBADEB822FE
:0B146600DFBFDEBD908002E523F02216
:101B0600EE2F60250E908000E521304204C2E18070
:101B160007C2E0121F8A6403121F8A6403121F8A17
:0A1B2600D2E0121F8ADFE3DEE122A5
:101ADB00A2469240C2461212E9EE2F60140E90807D
:101AEB0000E5216403121F8A6403121F8ADFF4DEF0
:0B1AFB00F2121E7DC23BA24092462268
:101E7D00E523908002D2E4F07828121F6FC2E4F0BF
:051E8D007828021F6F20
:1012E900D3121DF5908000E521C2E1F07817121F95
:1012F9006F205025D2E0C2AFF0E523908002C2E012
:10130900F0D2AF780C121F6FD2E0C2AFF09080001C
:10131900E521C2E1F0D2AF8023D231E526908010D9
:10132900F0E523908002D2E1F0780C121F6FC2E140
:10133900F0C231E526908010F09080007812121FDB
:0A1349006FE521F0D23BC3021DF551
:101EF100908000E5216403121F8A6403121F8ADFA8
:021F0100F422C8
:0C1F6300908003E524C2E6F0D2E6F022F4
:101DF500E5254004D2E68002C2E6908004F0F52590
:081E05004001227805021F6F65
:021FFE000225BA
:0F1F4600C2AF908000E0E0D330E101C3D2AF2200
:1010E40090E781E054F0B4F0061215D1021169B40E
:1010F40000051211FC806EB410051219268066B426
:101104002005121621805EB43005121BCE8056B421
:101114004005121CCE804EB450051218458046B4CA
:1011240060081214CC121F14803BB470051218EF1F
:101134008033B48005121524802BB4900512127DDF
:101144008023B4A005121746801BB4B005120046D4
:101154008013B4C005121E0D800BB4D005121E0DF1
:0C1164008003120BCE90E68D7400F02288
:051F95007406021E0F9E
:051F9A007415021E0F8A
:101E0D007418C25690E095858353858254F0A3745F
:081E1D0000F0F54F75500122A1
:101D5800C25690E09585835385825474A5F0A3E517
:0F1D68003BF0540F240354FE03F550754F002237
:101F140090E0977462F53B7402F0A37425F0021DFF
:011F24005864
:101EA7007E007F0090E09774E2F53BEEF0A3EFF041
:031EB700021D58B1
:1015D100A3E0A3B403030216BDB40A030216BBB40D
:1015E1000003021F25B401030216BDB40203021653
:1015F100BFB40403021B58B4050302166EB40603FC
:1016010002157CB407030219C4B40805E0FF021EE9
:10161100BAB4090BE0FFA3E0FD1219F6021F9522EF
:101EBA00121B8090E09774F2F53B7408F0A3EFF0E0
:031ECA00021D589E
:101F2500121BA7E0F536FEA3E0F537FF052F021FCC
:011F35009516
:1016BB00052F052F121BA7E0FEF536A3E0FFF5372C
:1016CB00C3E54B9420E54A9400500A204C07E4B53F
:1016DB002F03021E0DD25690E782E0B40302800363
:1016EB00B40A0F7C0090E787E0FD14252FF52F122D
:0716FB001CF18E4F8F5022FD
:101B58007400F52FE54A454B601B304C0F90800010
:101B680078007900E030E104D8FAD9F8121F6375DB
:081B78004A00754B00021F95A5
:10166E00121BA7E0FCA3E0FDA3E0F8A3E0F9A3E0C2
:10167E00FAA3E0FB90E094ECF0E525D2E1D2E0BCD9
:10168E000306C2E0D2E18007BC0204C2E1D2E0F55B
:10169E0025908004F090E091EDF090E092E8F0A3B8
:0D16AE00E9F090E08CEAF0A3EBF0021F954C
:1019C40090E786E0FEA3E0FF90E783E0B4000D30EB
:1019D4003C05121ADB8010121B06800B303A0512EC
:1019E4001E678003121B30D230E526908010F0026F
:0219F4001F953D
:10157C00C230E526908010F090E784E0FF7E00A357
:10158C00A3A3E0FCA3E0FD121CF190E783E0B40000
:10159C0020303C08203B05C2461212E97C0790E73C
:1015AC0081E090E789540FB40802E0FC1214168015
:1015BC0011303A0B203E03121990121BF3800312C8
:0515CC001B30021F9519
:101BA70090E783E0B40009204E19D24E7D408007AC
:101BB700304E10C24E7D207F101219F67DD87F005F
:071BC7001219F690E78422D9
:100BCE00A3E0A3C3B40002804DB401028022B4029C
:100BDE00028044B403028019B40403021EA7B405B4
:100BEE00028067B40603020C7FB40703020C88224E
:100BFE00D3120C4D90E786500CE584F8E0A3F6086E
:100C0E00DFFA021F95C2AFE0A30586F0A30586DFCB
:100C1E00F6D2AF021F95D3120C4D90E097753BE8BC
:100C2E00500CE584F8E608F0A3DFFA021D58C2AFB7
:100C3E000586E0A30586F0A3DFF6D2AF021D58E0CD
:100C4E00FFA3E0F584A3E0F58522E0900C69F09017
:100C5E000C76F090E784E0FFC2AFE5A090E097F04D
:100C6E005F90E785FFE04FF5A0D2AF753BE1021D27
:100C7E005812000E121809021F95E0B40402801FCC
:100C8E005403C2AFF5512455F582E4341FF583E4C5
:100C9E0093F8E52454F048F524908003F0D2AF90F9
:0B0CAE00E097E551F0753BE1021D5896
:101E9200C390E6787800E020E003D8FA2220E2FC42
:051EA20030E1F9D3223C
:101D3600C2AF90E6787480F090E679EF54FEF01228
:101D46001E92500D7400F090E679EDF0121E92503E
:021D5600002269
:101C1800121D36500990E679EBF0121E92C390E639
:101C2800787440F0500890E679E0FF90E678E0207C
:051C3800E6FCD2AF2222
:101C8600121D36501B7480F090E679EF54FE440125
:101C9600F0121E92500A7420F090E679E0121E921D
:041CA600D3021C2623
:101CAA00C2A3C2A779C77B027A08E933F9C2A25054
:101CBA0002D2A2D2A3C2A3DAF1EF304201F4F9DBD5
:041CCA00E7D2A72294
:101A5500C2A3C2867A027400121A74EF304201F4EE
:101A65007A08121A747A067400121A74D28622330E
:0E1A7500F9C2A25002D2A2D2A3C2A3DAF22278
:10195B00C2A3C2A779A77A08E933F9C2A25002D26F
:10196B00A2D2A3C2A3DAF17840000000D8FB7A0818
:10197B007F00C372A4EF33FFD2A3C2A3DAF4D2A7C2
:05198B00E5342FFF22EE
:101D9400C2A3C2A77A0CC3D2A372A4EF33FFC2A317
:091DA400DAF4D2A7E5342FFF2286
:1019F600C2AFD2A0E520D2E4F5B1F520EFF97B0223
:101A06007A08E933F9C2A15002D2A1C2A0D2A0DA63
:101A1600F1EDF9DBEBE520C2E4F520F5B1D2AF221A
:1013B80090E6A2E020E108E5507005E54F700122B3
:1013C8007820E550C398E54F94005002A850E8F9FA
:1013D80085548485538574C0F59B74E7F59A90E627
:1013E8007BC2AF0586E0A30586F00586E0A30586E7
:1013F800F0D8F0D2AF90E68FE929F085845485853E
:0E14080053E550C399F550E54F9400F54F227F
:10135300000000E5BB20E70122304F1590E6D0E006
:10136300700E90E6D1E07008C24F90E6487402F028
:1013730022E5567005E555700122C3E556255690C2
:10138300E6D1F0000000E555355590E6D0F0740441
:10139300F5BBC3E54B9556F54BE54A9555F54AC361
:1013A300E5509556F550E54F9555F54F7006E550C8
:0513B3007002D24F2280
:011FB10032FD
:101055006080E00008013F01010101070100030074
:1010650000001000FFFEFEFFFFFFFFFF010900006B
:10107500002D123F0803013F010101070102040190
:1010850000000000FFFDFFFFFFFFFFFF090912122F
:10109500002D363F0E03013F010136070100020115
:1010A50000001100FFFEFEFEFFFFFFFF0009121208
:1010B500002D123F0803013F010101070102000154
:1010C50000000000FFFDFFFFFFFFFFFF09091212EF
:0E10D500002D363F47E080800000FF06E4114A
:1014710090E60174CAF090E6F574FFF090E080E028
:1014810090E6F3F090E081E090E6C3F090E082E036
:1014910090E6C1F090E083E090E6C2F090E085E054
:1014A10090E6C0F090E086E090E6F4F075AF077446
:1014B100E0F59A7400F59B759DE4E4F59EFF90E6D6
:0A14C1007BE090E67CF00FBF80F4A2
:0114CB0022FE
:100E5700C24BE55FB4061BE5636003020EF27563E0
:100E670006303903020EF25324F0908003E524F094
:100E77008079E5636075655F6071855F64E55F64D0
:100E8700076005E563B4060C756407D254C238756C
:100E97006538802CA2549238C254C3E55F9563F538
:100EA7006530E706F404F565D254E54E700AE5654A
:100EB70075F00CA4F5658008E56575F00EA4F56579
:100EC700C249755703E4F56390003D93F566E4F571
:100ED7005CE5515403901F5593FFE52454F0FEEF52
:0E0EE7004EF524908003E524F0C24DD24B223C
:03004300020F00A9
:03005300020F0099
:100F0000021DAD00021E3B00021E2500021DC50091
:100F1000021881000218B8000200520002005200BC
:100F2000021FB1000200520002005200021DDD004B
:100F30000200520002005200020052000200520061
:100F40000200520002005200020052000200520051
:100F50000200520002005200020052000200520041
:100F60000200520002005200020052000200520031
:100F70000200520002005200020052000200520021
:100F80000200520002005200020052000200520011
:100F90000200520002005200020052000200520001
:100FA00002005200020052000200520002005200F1
:080FB000020052000200520091
:101A830090E682E030E004E020E60B90E682E0306E
:101A9300E119E030E71590E680E04401F07F147E21
:0C1AA3000012178990E680E054FEF0224B
:101C3D0090E682E044C0F090E681F0438701000019
:041C4D000000002271
:101A260030610990E680E0440AF0800790E680E0A5
:101A36004408F07FDC7E0512178990E65D74FFF09E
:0F1A460090E65FF05391EF90E680E054F7F022C6
:021AAF00A90785
:101AB100AE4CAF4D8F828E83A3E064037017AD01EE
:101AC10019ED7001228F828E83E07C002FFDEC3EA8
:091AD100FEAF0580DF7E007F00FE
:011ADA0022E9
:101789008E188F1990E600E05418700DE518C313F0
:10179900F518E51913F519801590E600E05418FFBE
:1017A900BF100BE51925E0F519E51833F518E5190A
:1017B9001519AE18700215184E6005121C5180EEED
:0117C90022FD
:101C51007400F58690FDA57C05A3E582458370F9A6
:011C61002260
:030000000211707A
:0C117000787FE4F6D8FD7581660211B7A7
:101CF100EF8DF0A4A8F0CF8CF0A428CE8DF0A42E07
:021D0100FE22C0
:101D0300EB9FF5F0EA9E42F0E99D42F0E89C45F036
:011D130022AD
:10117C00020675E493A3F8E493A34003F68001F20E
:10118C0008DFF48029E493A3F85407240CC8C33374
:10119C00C4540F4420C8834004F456800146F6DF43
:1011AC00E4800B0102040810204080901055E47E6E
:1011BC00019360BCA3FF543F30E509541FFEE49338
:1011CC00A360010ECF54C025E060A840B8E493A3FF
:1011DC00FAE493A3F8E493A3C8C582C8CAC583CA2A
:1011EC00F0A3C8C582C8CAC583CADFE9DEE780BEE2
:0110E300000C
:00000001FF
